:100000000C945A000C9477000C9477000C947700B1
:100010000C9477000C9477000C9477000C94770084
:100020000C9477000C9477000C9477000C94770074
:100030000C9477000C9477000C9477000C94770064
:100040000C94EB010C9477000C9477000C947700DF
:100050000C9477000C9477000C9477000C94770044
:100060000C9477000C947700000024272A000025C8
:10007000282B000023262904040404040404040299
:100080000202020202030303030303010204081035
:100090002040800102040810200102040810200002
:1000A0000000070002010000030406000000000039
:1000B0000000000011241FBECFEFD4E0DEBFCDBF93
:1000C00011E0A0E0B1E0ECECF7E002C005900D9289
:1000D000A231B107D9F711E0A2E1B1E001C01D9250
:1000E000AA31B107E1F70E94E4010C94E5030C94F6
:1000F0000000EF92FF920F931F93CF93DF938091B5
:1001000000010E942C038C01809102010E942C03AB
:100110007C01809104010E942C03EC018091060176
:100120000E942C0360E070E0012B11F461E070E0AC
:1001300020E030E0892B11F421E030E0220F331F62
:1001400040E050E0CD2B11F441E050E0240F351F8A
:10015000220F331F40E050E0EF2811F441E050E05F
:10016000240F351F220F331FCB01820F931FDF9106
:10017000CF911F910F91FF90EF90089560E070E094
:1001800080910E010E94BA0260E070E080910C0143
:100190000E94BA0260E070E080910A010E94BA02F7
:1001A00008956FE170E080910E010E94BA026FEF36
:1001B00070E080910C010E94BA0260E070E08091D2
:1001C0000A010E94BA02089560E070E080910E0179
:1001D0000E94BA0262E370E080910C010E94BA02B0
:1001E0006FEF70E080910A010E94BA02089567EFF4
:1001F00070E080910E010E94BA026CE170E0809183
:100200000C010E94BA0266EB70E080910A010E9424
:10021000BA0208956FEF70E080910E010E94BA0259
:1002200060E070E080910C010E94BA0260E070E032
:1002300080910A010E94BA0208956FEF70E08091E8
:100240000E010E94BA0260E570E080910C010E94EC
:10025000BA0260E070E080910A010E94BA0208953B
:100260006FEF70E080910E010E94BA026AE570E0C3
:1002700080910C010E94BA0262E370E080910A0151
:100280000E94BA0208950E947900009719F40E9412
:10029000BE0008958130910519F40E941D01089552
:1002A0008230910519F40E940A0108958330910566
:1002B00019F40E94F70008958430910519F40E9402
:1002C000E40008958530910519F40E94D100089545
:1002D0000F9711F40E94300108950E9443016AE0D3
:1002E00070E080E090E00E942802089561E0809133
:1002F00008010E94780364E670E080E090E00E94CC
:10030000280260E0809108010E947803089560E06F
:10031000809100010E940E0360E0809102010E9422
:100320000E0360E0809104010E940E0360E0809162
:1003300006010E940E0361E0809108010E940E03F5
:1003400061E080910E010E940E0361E080910C013A
:100350000E940E0361E080910A010E940E030E9438
:10036000300168EE73E080E090E00E9428020E9475
:100370001D0168EE73E080E090E00E9428020E9478
:100380000A0168EE73E080E090E00E9428020E947B
:10039000F70068EE73E080E090E00E9428020E947F
:1003A000E40068EE73E080E090E00E9428020E9482
:1003B000D10068EE73E080E090E00E9428020E9485
:1003C000BE000E94760108950E9457020E94870194
:1003D0000E946D01FDCF1F920F920FB60F92112454
:1003E0008F939F93AF93BF938091160190911701C4
:1003F000A0911801B09119010196A11DB11D809322
:10040000160190931701A0931801B0931901BF91A1
:10041000AF919F918F910F900FBE0F901F901895E5
:100420006091160170911701809118019091190146
:1004300027E0660F771F881F991F2A95D1F72DE7B0
:1004400030E040E050E00E94C303CA01B9010895C2
:10045000AF92BF92CF92DF92EF92FF920F931F93D2
:100460005B016C010E9410027B018C010E94100252
:100470006E197F09800B910B6A157B058C059D0514
:10048000A8F31F910F91FF90EF90DF90CF90BF9056
:10049000AF900895019751F0880F991F880F991F09
:1004A00002972FB7F8940197F1F72FBF089578942A
:1004B0001092160110921701109218011092190152
:1004C00084B5826084BD84B5816084BD85B5826059
:1004D00085BD85B5816085BDEEE6F0E080818160F7
:1004E0008083E1E8F0E080818260808380818160A8
:1004F0008083E0E8F0E0808181608083E1EBF0E0E0
:10050000808184608083E0EBF0E080818160808383
:10051000EAE7F0E08081846080838081826080836C
:100520008081816080838081806880831092C10097
:100530000895809310010895909110019295990F5C
:10054000990F907C8F70982B90937C0080917A000B
:10055000806480937A0080917A0086FDFCCF2091A0
:100560007800809179009927982F88273327822B4C
:10057000932B08951F93CF93DF93182FEB0161E026
:100580000E940E03E12FFF27E156FF4F8491833035
:1005900051F480918000806880938000D09389001E
:1005A000C093880037C0843051F48091800080620D
:1005B00080938000D0938B00C0938A002BC0813041
:1005C00029F484B5806884BDC7BD24C0823029F475
:1005D00084B5806284BDC8BD1DC0863041F4809161
:1005E000B00080688093B000C093B30013C0873020
:1005F00041F48091B00080628093B000C093B40059
:1006000009C0C038D10514F460E001C061E0812F59
:100610000E947803DF91CF911F910895282F3327EF
:10062000C90185579F4FFC01949129583F4FF9010B
:100630008491882381F0E82FFF27E859FF4FE49148
:10064000FF27662329F4808190958923808308956C
:100650008081892B80830895482F5527CA018156B0
:100660009F4FFC012491CA0185579F4FFC01949133
:1006700049585F4FFA013491332319F480E090E038
:100680000895222331F1233021F4809180008F7767
:1006900005C0243031F4809180008F7D80938000EC
:1006A00018C0213019F484B58F7704C0223021F4AA
:1006B00084B58F7D84BD0DC0263021F48091B000BB
:1006C0008F7705C0273029F48091B0008F7D80930B
:1006D000B000E32FFF27EE58FF4FE491FF27808102
:1006E00020E030E0892311F021E030E0C9010895D5
:1006F000482F5527CA0181569F4FFC012491CA01FA
:1007000085579F4FFC01949149585F4FFA013491EE
:100710003323C1F1222331F1233021F48091800071
:100720008F7705C0243031F4809180008F7D8093D5
:10073000800018C0213019F484B58F7704C02230AE
:1007400021F484B58F7D84BD0DC0263021F48091C5
:10075000B0008F7705C0273029F48091B0008F7DDD
:100760008093B000E32FFF27E359FF4FE491FF2769
:10077000662329F480819095892380830895808160
:10078000892B80830895A1E21A2EAA1BBB1BFD01B1
:100790000DC0AA1FBB1FEE1FFF1FA217B307E40760
:1007A000F50720F0A21BB30BE40BF50B661F771FB8
:1007B000881F991F1A9469F7609570958095909598
:0C07C0009B01AC01BD01CF010895FFCFEB
:1007CC000200030004000500060009000A000B00EB
:0207DC0001001A
:00000001FF
